:030000000208AA49
:080003000280038E828F83222C
:08000B0002800BAE82AF8322DC
:08001300028013742D0173003B
:08001B0002801B11730171004A
:08002300028023111601710097
:03002B0002802B25
:10002E00217601730167216521872194018A01CE12
:10003E0021CE21A802092A020A85017D0201BB02F6
:10004E0009CE0209D4020A1202086B020831020715
:10005E00BC02079202094D214A3098FDC298E599DB
:10006E0022117174203099FDC299F59922117DC02B
:10007E00E0740D1173740A1173D0E022C2D51162AF
:10008E0031A8B41B03D3E422B40D05D2D5C3E422A8
:10009E00FA314A40E9CA1173116231A8B41B0280C9
:1000AE00E4B40D03EAC322B40804117380D0B4156E
:1000BE000280F7FB314A40E0CB1173EAC44BC322F6
:1000CE007A007B007C04C2D5116231A8B41B07D321
:1000DE00E4F583F58222B408028003B47F0CBC04DD
:1000EE000280E5117331390C80DEB40D108B838ADA
:1000FE0082BC0407E4F583F582D2D5C322FD314AD2
:10010E0040C6CD120073EDC0E03128D0E02AFAE4EB
:10011E003BFBDCB4C38A828B8322EBC454F0FBEA34
:10012E00C4540F4BFBEAC454F0FA22EAC4540FFA3B
:10013E00EBC454F04AFAEBC4540FFB22C324D05044
:10014E001424F64004240AC32224F9500824FA4049
:10015E00042410C322D322C0E0C4540F24F650024C
:10016E002407243A1173D0E0C0E0540F24F6500255
:10017E002407243A1173D0E022C0E0E5833165E50F
:10018E00823165D0E022C0E0E493A3600AA2E75476
:10019E007F1173400280F1D0E022C0E0C394614031
:1001AE0009941A5005D0E024E022D0E0227800C055
:1001BE00E0E4936008A2E7084003A380F4D0E022B5
:1001CE00C0E0C3309808E599B41B01D3C298D0E0C3
:1001DE0022900D213194EF3165EE3165319411622B
:1001EE0031A875F0DFC0F075F001C0F0F5F0901099
:1001FE0000F1925024758204E493B4FE150582E456
:10020E0093B5F00E11717582203194117D75824077
:10021E00E4730583E583B400D8E5F0B43F07900E90
:10022E00871145A1D6B44D07900E8F114581C6B4E6
:10023E005207900E941145A13DB44C07900ECE314D
:10024E009441A8B45507900E9B1145C14BB44E076F
:10025E00900E9E1145E13DB44A07900EA2114581C4
:10026E0014B44807900EA81145814BB44507900E63
:10027E00B41145818CB44307900EB91145E119B400
:10028E005A0B74006012900EBD1145E14DB4490831
:10029E00900EAE1145020773017D900DB911457890
:1002AE00107A10760008DAFB1167B41B028074B462
:1002BE003A0679007143800A314A40EC790671435F
:1002CE0080E67C007162F87162F5837162F582716D
:1002DE0062B40104D29780317026E860187162FA18
:1002EE0079017143EAA2E7929712086BE43402F99E
:1002FE007143A3D8E57162EC60AE7904714380A8B6
:10030E00E860F27162D8FC80ECE860047162D8F3A8
:10031E007162EC70E5713A900DD8114530987A11F2
:10032E00678076713A900DD01145806D7800790016
:10033E00D9FED8FA22E95407232410F907E77002F0
:10034E00090722D3878209878309E5827005E58331
:10035E007001C322116731A8B41B06D0E0D0E08033
:10036E00C2B43A0A79057143D0E0D0E041D0314AA7
:10037E0050067907714380DCFA116731A8B41B026D
:10038E0080D9B43A0280DD314A5006790771438034
:10039E00E8CAC44AFA2CFCEA22EEC0E0EFC0E090B4
:1003AE000DDF114579107EE87F0D91107EEE7F0DE9
:1003BE0091107EF37F0D91107A0571514009DAFA92
:1003CE00900E2F11458025900DFE114579167E0257
:1003DE007F0E91027E137F0E91027E1B7F0E910285
:1003EE007E217F0E91027E267F0E9102D0E0FFD0FD
:1003FE00E0FE017D715150091171120A12110611A0
:10040E004522715180F2900D601145110631879091
:10041E000D2E114511CE20D5065002E114110E11EC
:10042E007D900E3D11451106E4F5D0F5F0F8F9FA80
:10043E00FBFCFDFEFF758108C0E0C0E0737A101171
:10044E007B11063187743A111E7B101106E493A3BB
:10045E0031651171DBF7116F7B101106E493A35414
:10046E007FB47F01E424E04001E424201173DBEC2F
:10047E00117DD1D0110E31CE4002DAC5017D900D25
:10048E00A2114511CE110E117D3187743A111E74D1
:10049E00281173110EE4933165900D7B1145118A6D
:1004AE0020D510400E110612086B117D1106A311F6
:1004BE000E8197900DAE0145900D6A11457815117C
:1004CE0071D8FC1145758310F1924002017D116FB8
:1004DE00758220319475822031BB7421C398F874D3
:1004EE00201173D8FC758200318778067420117341
:1004FE00D8FC758204E493AA83B4FE05900E758031
:10050E0018B4FD05900E7C8010B42305900E7980F2
:10051E0008B4F90280EE900E8311458A83117D7422
:10052E00FFB5830281DA0583E583B4009B81DA117E
:10053E007B7AFF90100015830583E583B40002805B
:10054E0021F192501D758204E4934403F460E91185
:10055E006F0A74412A111E11267582203194117D65
:10056E00A146BAFF05900D370145900D291145742E
:10057E00411173111674412A1173900D2E114511EC
:10058E0062B41B02017DFB741FC39AEB400231A8BB
:10059E001173FB117DEBC3944140CFFBEAC39B402B
:1005AE00C90B90100015830583E583B400028017F4
:1005BE00F1925013758204E4934403F460E9DBE78F
:1005CE00117D758240813622900E5D11457C3F90E3
:1005DE000E8AD1407C4DD1407C52D1407C4CD140D2
:1005EE007C55D1407C4ED1407C4AD1407C48D14094
:1005FE007C49D1407C45D1407C43D140740060049D
:10060E007C5AD140900E6B1145901000F192502003
:10061E00758204E493B4FE11116F0582E493117395
:10062E0011267582203194117D0583E583B400DC9B
:10063E00017D116FEC117311261145017DD1E290F0
:10064E000E471145EB3165EA31651145ED3165EC2B
:10065E003165117D8D838C82A3AC82AD83900D5656
:10066E0011451167B41B02E112117D8A828B83EC56
:10067E00C39582FAED95837009EA603254F07002E8
:10068E0080027A10743A1173EA31653187E5832559
:10069E00822AFBE43165E49331652BFBA3DAF7EB99
:1006AE00F4043165117DD1D031CE50C38056743AE9
:1006BE001173E431653165316504316574FF31655F
:1006CE00017BE8C0E0780CE58C04000070FBD8F7E5
:1006DE00D0E0F822117B900D84114511CE402120DF
:1006EE00D51EC083C082117D900D8E114511CEADE9
:1006FE0083AC82D0E0FAD0E0FB400520D502017D2C
:10070E00D0E0D0E0117D900D190145D1E2900D9809
:10071E001145116231A8B459EB117B8B838A82E4A7
:10072E0012086BEDB58305ECB5820122A380F09023
:10073E000D4D114511CE40CE20D5CB110E017B11A2
:10074E007B900EBD1145742C111E900D9811451104
:10075E006231A8B459AE117B1207BC900EC2500381
:10076E00900EC90145117D7800117DE83165743A0E
:10077E0011731171E6316508E8540F70F5117DB8EB
:10078E0000E9017D758200E493B4A517A3E493B448
:10079E00E511A3E493B4E00BA3E493B4A50575822D
:1007AE0000D32274FFB58302C322058380D6740062
:1007BE006038908000E493F4700DA37400B582F558
:1007CE007400B583F0C322908000E4936006E412B7
:1007DE0008314016A37400B582F07400B583EB9017
:1007EE0080007CE87D04DC04DD02D3227420A2AFFD
:1007FE0092D1C2AFF0F07B147AE5DAFEDBFA74A088
:10080E00F07A05DAFEE493A2D192AFF470D8A37415
:10081E0000B583EA7400B582E574FF908000F0E4C1
:10082E00F0C322F5F0EAC0E0EBC0E07A197440A202
:10083E00AF92D1C2AFF0E5F0F07B13DBFE74C0F0E7
:10084E007B05DBFEE493A2D192AFC395F06003DA91
:10085E00DCD3E4F0D0E0FBD0E0FAE5F022C0E0C05B
:10086E00F0F5F07400601BE583B4FF02800B5012AC
:10087E00B48002800450028009E5F01131D0F0D02E
:10088E00E022E5F0F0E493C395F06009E0C395F043
:10089E006003D38001C3D0F0D0E02232E4F5A8F596
:1008AE00B875D00011A911A9F4F580F590F5A0F551
:1008BE00B075813079C87AF9DAFED9FA740060130E
:1008CE0074B5600F78FAA2B579C8D9FE4005D8F68E
:1008DE001207BC75F0F911FD312A75F0FD11FD906E
:1008EE000EE212019412007D7E007F800201DF90E5
:1008FE0010001207925024758204E493B5F015C0CF
:10090E00F0C083741EC0E07409C0E0758240E473C9
:10091E00D083D0F00583E583B400D72274FAF57B3B
:10092E00F57AF579F578637A556379CC63781DF5A8
:10093E008DF58B758921758780759852D28E2230F0
:10094E009806120067B41B51120067B41B4B31BBE3
:10095E00209803741B22120067B45B4431BB30989D
:10096E00DE120067B44103740B22B44203740A22F0
:10097E00B44303741522B44403740822B4350280C0
:10098E0007B4360280028018C0E031BB30980B12DB
:10099E000067B47E09D0E024E422D0E080A1D0E04C
:1009AE0031BB30989A120067B41BF580A1EAC0E003
:1009BE007A14E58C2098050470FADAF6D0E0FA2263
:1009CE00C0F0C0E08013C0F0C0E030E70C742D1210
:1009DE000073D0E0C0E0F4240175F06484D2D560D9
:1009EE0007C2D52430120073E5F075F00A8430D5B5
:1009FE000260052430120073E5F02430120073D02B
:100A0E00E0D0F022C0E0E8C0E0C2D5AA82AB837C81
:100A1E00107D27517060072430120073D2D57CE808
:100A2E007D035170700330D5072430120073D2D578
:100A3E007C647D005170700330D507243012007332
:100A4E00D2D5EAABF075F00A84700330D5052430A8
:100A5E00120073E5F08BF02430120073D0E0F8D062
:100A6E00E022780008C3EA9CFAEB9DFB50F618EAE8
:100A7E002CFAEB3DFBE822C0E0E8C0E0E9C0E0EC78
:100A8E00C0E0D2D1D2D5E493A3602520E72E547FC7
:100A9E00B40D0712007DD2D180ECB41F04C2D580F4
:100AAE00E5B40E0512007D8007C2D112007380D608
:100ABE00D0E0FCD0E0F9D0E0F8D0E022547FF8206E
:100ACE00D103120071C2D1C082C083900B3F7C0053
:100ADE00E86007F9712E70FCD9FA712E603CB40FE4
:100AEE0012712E0483801E68667767796278766B42
:100AFE00716A7A0483800E657461726E69736F6CAD
:100B0E00756D706463A2D592E5D2D5B81402C2E5B4
:100B1E00B80C02C2E512007380C0D083D08241941B
:100B2E00E493BC00057CFF540F227C00A3C4540F39
:100B3E00228290E82386054CF844B3B0B1485FF0AA
:100B4E00117FA0157F1C2ED1405A50F103BFBA0C55
:100B5E002F96018D3F95380D6F5F1207710E562F30
:100B6E00483B6258201F7670322440B840E1618FB6
:100B7E0001340BCA89D3C0A3B9588004F80285602A
:100B8E002591F092731F107F12549310444807D191
:100B9E0026564FD0F66472E0B83BD5F0164F56305D
:100BAE006F48025FA8201F017630D5602541A42C26
:100BBE0060056F013F261F30078E1DF06399F042CE
:100BCE00B8201F2330027AD1602FF0F6058F931ACA
:100BDE005028F082046FA30D3F1F514023013E05A4
:100BEE0043017A01176493302A088C243099B0F3AC
:100BFE001960254135098ECB191230051F311D04A0
:100C0E00144F761204AB279056012FA8D5F0AA26C2
:100C1E00205F1CF0F361FE0141730127C1C0848F78
:100C2E00D6018770564F19701FA8D99076021743B8
:100C3E00FE01C1840B157F028B14308F63396F193F
:100C4E00F011C9106D023F91097A41D0BA0C1D39CD
:100C5E005F07F2111720416B3509F775120BA7CC00
:100C6E0048023F6412A00C27E39FC0147770114016
:100C7E007121C0682541F0627FD1D021E16258B068
:100C8E00F3051F733077B16F19E01943E0582FF653
:100C9E00A414D02303FE31F5143099F8033F6422D7
:100CAE00516025412FE30156279309FE11FE79BAB3
:100CBE00607542EA6258A0E51F534FD1C0A30942A6
:100CCE0053F71204621B30F505F7690C351B708261
:100CDE002F2F144F51C064250057656C636F6D65DF
:100CEE008094322C2062791FF81FFE0D0E202053A7
:100CFE00656594322E444F432C94322E455155A4A3
:100D0E0094322E484452B4D58D2E0E201F9E1FA015
:100D1E00210D0E414444523A003EA086CA8228005C
:100D2E00292C958C80C83A20001F9782C373C7A6C2
:100D3E00832CBA204A554D508086A172820D0E0D1D
:100D4E000D1F8783813A20001FE4FB206B65793AE3
:100D5E0020000D0D1F888083812028000D0D1F821D
:100D6E001FFD001F8120202020201FC90E29201FBB
:100D7E00871FB23A200046697273741F813A2000B1
:100D8E004C6173741F813A2020001FB9A120737526
:100D9E0072653F000D0D416464726573733E2000F1
:100DAE0020201F9CC12C8E81F70D0E0D0D1F9F2034
:100DBE006173636969F9961F9884892C958C80A05C
:100DCE000D0E0D1F8AA065640D0E0D1F8AC1640DD8
:100DDE000E53756D6D6172793A0E20C67391640E65
:100DEE00208B91640E208B207772697474656E0E61
:100DFE001F9B3A0E208B20756E61626C658020778A
:100E0E00726974650E2020626164F5730E20859FF1
:100E1E0096C60E2085849D0E2085206E6F6E849D55
:100E2E000E1F979B2064657465637465640D0E0DCB
:100E3E00866E696E67823A0D0E0D0D53656E64698E
:100E4E006E671F988489AC20200020802020000D22
:100E5E000D5374616E646172641F9E730E1FDA1FF0
:100E6E00F465641F9E730E1F9A9E001F82001F8FD3
:100E7E001FE21FAA003F3F3F001FD7001F8ED7D192
:100E8E00001FD18273001F8682001F8A001F9300ED
:100E9E001F8781001F88808381001F84DB9A830057
:100EAE001F84DBC083001F9C9A92001FED83001FDE
:100EBE00CB9990001F9990CB640D0E1F859B0D0E44
:100ECE004C6F616420496E74656C2068657820668D
:100EDE00696C65000D0A0A4D544B3531203830359A
:100EEE0031204D4943524F434F4E54524F4C4C4577
:100EFE005220545241494E4552204B49540D0A003E
:10100000A5E5E0A5FE44000000000000000000008F
:10101000000000000000000000000000FFFFFFFFD4
:0F102000446973617373656D626C65000200480B
:10104000112C7D14C2D1114CDDFC012CEFF5835124
:101050004FEEF582514FE493FAA3E493FBA3E4939C
:10106000FCEA5408700FEA035478F8EA54074890F1
:1010700016C8938008EAC4540F901362935403F87F
:101080002EFEEF3400FF743A512A719D20D121EADF
:10109000514F719DB80104790B8011EB514F719D37
:1010A000B8020479088005EC514F7906719DD9FC8E
:1010B000EA54087010901748EA035478F8EA540785
:1010C0004893F980099017C8EAC4540F93F9901E09
:1010D000947808C374204007E99309A2E7547F512C
:1010E0002AD8F1741BC0E07411C0E0EA5408700FF4
:1010F000EA035478F8EA5407489016C8938008EA3F
:10110000C4540F9013629354FC03031490111D23D5
:101110002582F582E43583F583E473012C412D416A
:101120003C21812172414841044152415821A22170
:10113000D7415E4169416D4108411021AA218321B7
:101140007441714177417D413E411C418121DF4124
:101150001441C54185418B41914195419B41A94134
:10116000AF41B541BB410C41BF41CB41D741E74104
:10117000ED2231F67440512A7452512AEA54014149
:101180004531F6EB20E703EB414F9012F5E493A3D2
:1011900060F5F8C39B7003020038E493A330E7FACC
:1011A00080EB511031F8742F512AEB547823C4F896
:1011B000EB54806014901372E893901F293582F5E8
:1011C000825002058331978005E82420514F742E08
:1011D000512AEB5407414531F6318331F8ECFBEBF2
:1011E0002EF582EB20E703E48002E4F43FF583026E
:1011F00000367440412A5108742C512A7420412A27
:101200007423412A318331F87441412A31AA31F8DB
:101210007443412A31F25108742B512A7444512AE3
:101220007450512A7454512A7452020030EF54F809
:10123000F8EAC403540748514FEB414F31F674525A
:10124000512AEA540702002E510831F85100EB02EE
:1012500000343183ECFB414A511031F821AA510886
:1012600031F85100EB514F21DB513E416031744167
:101270006051087442412A513E31F821DF31832107
:10128000DB31AA21DB513E31F84108513E31F821D2
:1012900083513E414A318331F8413EEBC0E0ECFBE3
:1012A000318331F8D0E0FB2183318331F82174316F
:1012B0007431F84108317431F821833174414A5155
:1012C0001C31F85100EB514FEC414F31F631F251E6
:1012D00008742B512A411C31F631F25108742B51FC
:1012E0002A7450512A411031F631F2411C31F25129
:1012F0001C31F84108E04143C38153D0824450CCB3
:10130000834450C88050B09050B1A050B2B050B398
:1013100099534255C6CD5448B2C85432434FCECCEF
:10132000544CB2CB5243415032C8CA52434150325E
:10133000CC8C5448B08A544CB08D5448B18B544C2A
:10134000B1F0C2D05053D7A849C5B849D089544D3F
:101350004FC48854434FCE9853434FCE8750434F8A
:10136000CE00595909090909097A7E0976330952CB
:101370000971000206080C0E101214161B1E202301
:101380002425F8F0E493C398227950E58DF404F80D
:10139000D8FED9F722514F743A412A514F74204157
:0113A0002A22
:10140000A5E5E0A5FE53000000000000000000007C
:10141000000000000000000000000000FFFFFFFFD0
:0C14200053696E676C652D537465700095
:1014400030B306901D1B020045900013E49324FE68
:101450006005901D3E8146A393F8E4A393F582882E
:101460008374027182700EA3741471827007A37466
:10147000EF71826011A882A983901D4B9146E951BA
:101480004FE8514F012CE5B85404F5B8901CFE917B
:1014900046EF514FEE514F901CE8914612003C2010
:1014A000D50D5007901D073197012CAE82AF83C236
:1014B0008A901D5A9146901E523197E4758108C05A
:1014C000E0C0E08E828F83F5D0F8F9FAFBFCFDFED8
:1014D000FFF5F0757CDD757D14D2AAD2AF737189EA
:1014E000D0E0F9D0E0F8D082D083D0D0D0E032C0C4
:1014F000E0C0D0C083C082E8C0E0E9C0E07189D21A
:1015000099719D719DE58124FBF8E6719BE5F07171
:101510009B08E62354015145719D08E6514F08E6AA
:10152000719B719D08E6719508E67195EA7195EBDE
:101530007195EC7195ED7195EE7195EF719B719DC3
:10154000E824F8719B719D719DE57C8E7CFEE57DA4
:101550008F7DFFEAC0E0EBC0E0ECC0E0D2D1114CDF
:10156000D0E0FCD0E0FBD0E0FAAF7DAE7CE581249A
:10157000F9F8E6F57C08E6F57D120062120040B449
:101580000D0281DEB4200281DEB43F07901DCB91B5
:1015900046A179B45113901E4B3197C2AA71897537
:1015A000080075090075810932B44802A1CDB45212
:1015B00002A1FDB45302C167B44102C1AAB42E070F
:1015C000901E523197A179A179743D412A901D99BD
:1015D0003197E47195719DA88118E6719B08E651D9
:1015E0004F7802790EA1ECE871957910719DE65162
:1015F0004F08D9F8112CB800EE112CA179901344A2
:101600003197B1C9E58124FCF8E6719B901348A895
:10161000A8D16090134BA8B8D16090134EA889D17F
:1016200060901353A888D160901358A898D1609007
:10163000135DA887D1607454512A7430512AB1C9FE
:10164000E58C514FE58A514F719D7454512A743184
:10165000512AB1C9E58D514FE58B514F112CA1791C
:101660003197B1C9E8619B7817719DD8FC901D81B5
:101670003197E58124F9F8E68E7CFE08E68F7DFF40
:10168000EAC0E0EBC0E0ECC0E0D2D1114CD0E0FC0D
:10169000D0E0FBD0E0FAE58124F9F8EEAE7CF57CF1
:1016A000F608EFAF7DF57DF6A179E58124FBF89092
:1016B0001DBB319712003A400820D505F6112CA128
:1016C00079901D073197A179AD066F39394649499F
:1016D00063066F39394649496306AD39160E111153
:1016E0006306AD39160E111166061A1F160E11117A
:1016F00066061A1F160E111166061A1F160E111114
:1017000066062269161F9292660622A14D8386867E
:101710009B06969D160E11112606225D4DAD8E8EEE
:101720002606423D2F2B37374606423D390E111112
:101730004606423D39571111A5061111390E1111F6
:10174000A9068989391A89895A0E48732B2B2B2BA4
:1017500030004375212121212E0E676E06060606F4
:1017600038006A700A0A0A0A330E5D5D5D5D5D5DD0
:101770003B00121212121212410E8F8F8F8F8F8F19
:101780003E005D354C4C4C4C7C0E124F244C4C4C66
:101790004C004C4F808080805D0E4C2B57924C4CFF
:1017A00012001C1C15151515630E191984888888DC
:1017B000600078781F278B8B530E5353194C4C4C79
:1017C000530053531C4C4C4C2B21060A5D128F4C7A
:0817D0004C804C1588274C4C9D
:10180000A5E5E0A5FDFF00000000000000000000CD
:10181000000000000000000000000000FFFFFFFFCC
:0F182000454550524F4D20626F6F74696E6700DF
:0A184000900200E030E001229175F3
:10190000A5E5E0A5FE510000000000000000000079
:10191000000000000000000000000000FFFFFFFFCB
:0B192000517569636B20686F6D6500F6
:071940007E007F8002102CE5
:10195400C0D0C0E012004890197C120038D0E012C8
:10196400003412004890198B120038D0D0E5D01200
:101974000034120048020000416363756D756C61A8
:10198400746F72203D2000505357203D2000FEEB21
:10199400A4FD8EF0ECA4FCEB8EF0A4C5F02C2DC5B8
:1019A400F022E4FBFCFFE709B42D030FE709C3941D
:1019B40030B40A005012FA740A75F0001219922A0F
:1019C400FBE5F03400FC80E4EB8CF0DF002279705E
:1019D400120032B40D08770079701219A622B408E7
:1019E400061200301980E9B40C061200300980E0B8
:0719F400120030F70980D951
:101A0000A5E5E0A5FE5A000000000000000000006F
:101A1000000000000000000000000000FFFFFFFFCA
:0B1A20005A415020454550524F4D00E8
:101A4000901A6A120038743E120030120032B4311B
:101A500004718F80EBB43204712F80E4B4330491AD
:101A60007580DD7E007F8002102C0D0A32344C43DD
:101A700032353620454550524F4D2066756E6374A1
:101A8000696F6E73203120534156452C203220441B
:101A9000554D502C2033204C4F41440D0A00D2B4F8
:101AA000D2900000C2B40000C290227F083392B4EA
:101AB0009297D29000000000C290DFF1D2B4D29091
:101AC00000000000A2B4C290227F08D29000000063
:101AD00000A2B4929733C290DFF122C2B4D2900038
:101AE000000000C290D2B422C2B4D2900000000024
:101AF00000D2B422519E74A051AB40F822519E7482
:101B0000A051ABE58351ABE58251AB519E74A1511D
:101B1000AB51C951E822F5F0519E74A051ABE58359
:101B200051ABE58251ABE5F051AB51E851F4229055
:101B30001B5D12003812003C1200487A1012004857
:101B400012003674201200307B1051FDA3120034B5
:101B50007420120030DBF3DAE4120048220D0A652B
:101B60006570726F6D2061646472657373205B30A1
:101B70003030302D374646465D203E200074012629
:101B8000F608740036F622E6F58208E6F583229020
:101B90001C2312003812003C500122E582AA83C0A7
:101BA00083C0829000007116900001EA7116D08205
:101BB000D083787EE582F608E583F6901C42120019
:101BC000381219D2F4F582E5F0F4F583A312004837
:101BD000C083C082E582AA83900002711690000340
:101BE000EA7116D082D083787C7410F6087400F6FF
:101BF000C083C082787E7187E0FB787C7187EB714F
:101C000016787E717D787C717DD082D083740D12C0
:101C10000030120053A3E583458270D4901C6D12EE
:101C20000038220D0A536176652050726F67726129
:101C30006D20737461727420616464726573733EA5
:101C400020000D0A4E756D626572206F6620627904
:101C5000746573205B302D33323736385D203E207B
:101C6000000D0A536176696E672E2E2E000D446FAB
:101C70006E652E2E00901CDB12003890000051FD86
:101C8000787EF690000151FD787FF67410787CF62E
:101C9000087400F690000251FDFA90000351FDF522
:101CA000838A82C083C082787C718751FDFB787EF5
:101CB0007187EBF0787E717D787C717DD082D083E6
:101CC000A3E583458270DC90000051FDFA9000018D
:101CD00051FDF5838A82C082C083220D0A4C6F6158
:101CE00064696E672E2E2E00292C206F72203C45D1
:101CF00053433E20746F20657869743A20000D1FAD
:101D00008880838120280020436F6D6D616E642080
:101D100041626F727465642E0D0A000DA1C52063C7
:101D20006F6E6E65637420494E5431202870696E61
:101D300020313329206C6F7780BACFCC0D009432DC
:101D4000B3C7AE8120303031330D001FB8B3FFA5CB
:101D500020766563746F72AE20000D4E6F77866ECD
:101D6000696E67A6CFCC206D6F64653A20203C5227
:101D700045543E3DCC2C203F3D2048656C700D0DF8
:101D800000536B697070696E6720496E7374727569
:101D90006374696F6E2D3E20000D0A4C6F633A200C
:101DA00020496E742052414D204D656D6F7279202F
:101DB000436F6E74656E74730D0A004E6577204133
:101DC00063632056616C75653A20000D1FCF1FCCF0
:101DD0001F9E3A0D3C5245543E2086D4F60D203CC1
:101DE00053503E2086D4F60D20273F272020FF8E1B
:101DF000D70D20272E272020FFC4FD730D2027524A
:101E0000272020FF207370656369616C2066756E02
:101E10006374696F6EC4730D20274827202084DB0C
:101E2000C0920D202753272020FCD4F60D202741F7
:101E3000272020F0A2204163632076616C75650D38
:101E4000202751272020C8CFCC0D0E517569740D65
:101E50000A00202041434320422043204450545252
:101E6000202052302052312052322052332052341E
:101E70002052352052362052372020535020202027
:101E8000416464722020496E737472756374696F63
:101E90006E0D0A004143414CCC004144C400414412
:101EA00044C3414A4DD0414ECC434A4EC5434CD227
:101EB0004350CC44C14445C34449D6444A4EDA4910
:101EC0004EC34AC24A42C34AC34A4DD04A4EC24A8E
:101ED0004EC34A4EDA4ADA4C43414CCC4C4A4DD0C0
:101EE0004D4FD64D4F56C34D4F56D84D55CC4E4FF6
:101EF000D04F52CC504FD0505553C85245D4524574
:101F000054C952CC524CC352D25252C3534554C2FC
:101F1000534A4DD0535542C2535741D05843C858E5
:101F20004348C45852CC3F3FBF50B054434FCE50AB
:101F3000B153434FCE50B249C550B349D043B054CA
:0F1F400032434FCE5053D744B84143C3FDC2FE86
:20200000A5E5E0A5FE5700000000000000000000000000000000000000000000FFFFFFFF60
:0D2020004E455720434F4D4D414E44530057
:20204000758107902BBF79007AF07BD87C02EB4C601CE493A3CAC583CAC9C582C9F0A3CA76
:20206000C583CAC9C582C91BBBFFE31C80E090F2EBE4F012207690F000E0A3F5F0E0C5F0DB
:20208000C0E0C0F01227471581158112223A12279090F2E6F01225DF1220B112227F1223D4
:2020A000491223A912244312222012225002208E2290F2E6E0122AA97B61122AA0122B4470
:2020C00045F070030220DD749E75F0F0C0E0C0F0122747158115811220DE12223A2274D210
:2020E00075F0F0C0E0C0F012274715811581740290F2D8F090F2D8E075F0007B087C00121F
:202100002B5745F0700302213E800C90F2D8E00490F2D8F01480DD74DB75F0F0C0E0C0F0BB
:2021200090F2D8E075F000C0E0C0F0740275F000122736158115811581158102210B740A62
:2021400075F000C0E0C0F012275A1581158174E175F0F0C0E0C0F0122747158115817400F1
:2021600090F2D9F090F2D9E075F0007B0F7C00122B5E45F0700302221F800C90F2D9E0041D
:2021800090F2D9F01480DD74E575F0F0C0E0C0F090F2D9E075F000C0E0C0F0740275F000BA
:2021A0001227361581158115811581740290F2D8F090F2D8E075F0007B087C00122B574521
:2021C000F0700302221C800C90F2D8E00490F2D8F01480DD90F2D8E090F2DAF090F2DAE015
:2021E00075F0007B047C00122AF990F2DAF074EF75F0F0C0E0C0F090F2DAE090F2D9122B22
:20220000AD4B75F000C0E0C0F0740275F00012273615811581158115810221C802217B22C4
:2022200090F2E6E0122AA97B71122AA0122B4445F070030222390200002290F002E0A3F505
:20224000F0E0C5F0C0E0C0F0122747158115812290F2E6E0122AA97B0D122AA0122B444584
:20226000F0700302227E90F000E0A3F5F0E0C5F0C0E0C0F01227471581158112223A2290C0
:20228000F2E6E0122AA97B64122AA0122B4445F0700302234874F575F0F0C0E0C0F0122709
:2022A0004715811581740E75F0F1C0E0C0F01227471581158179DC7AF2E98AF0C0E0C0F063
:2022C000740A75F000C0E0C0F01227A2158115811581158179DC7AF2E98AF0C0E0C0F01212
:2022E00028031581158190F2E7F0A3C5F0F0C5F0742675F0F1C0E0C0F0740175F0001227DE
:202300003615811581743875F0F1C0E0C0F090F2E7E0A3F5F0E0C5F0C0E0C0F090F2E7E00A
:20232000A3F5F0E0C5F0C0E0C0F090F2E7E0A3F5F0E0C5F0C0E0C0F0740475F0001227362E
:202340007FF8122A8312223A2290F2E6E0122AA97B72122AA0122B4445F070030223A87457
:202360004875F0F1C0E0C0F012274715811581746675F0F1C0E0C0F079007A0289828A8336
:20238000E075F000C0E0C0F079007A0289828A83E075F000C0E0C0F0740375F000122736BB
:2023A0007FFA122A8312223A2290F2E6E0122AA97B69122AA0122B4445F070030224427463
:2023C0007275F0F1C0E0C0F012274715811581749275F0F1C0E0C0F012274715811581746D
:2023E000B375F0F1C0E0C0F01227471581158174D375F0F1C0E0C0F01227471581158174CB
:20240000F375F0F1C0E0C0F012274715811581741375F0F2C0E0C0F0122747158115817429
:202420003375F0F2C0E0C0F012274715811581745375F0F2C0E0C0F01227471581158112EA
:20244000223A2290F2E6E0122AA97B62122AA0122B4445F07003022515747A75F0F2C0E0CE
:20246000C0F012274715811581749975F0F2C0E0C0F01227471581158112260E90F2E9F0FF
:20248000A3C5F0F0C5F074AC75F0F2C0E0C0F012274715811581740090F2D8F090F2D8E0D4
:2024A00075F0007B107C00122B5745F07003022512800C90F2D8E00490F2D8F01480DD7442
:2024C000CA75F0F2C0E0C0F090F2E9E0A3F5F0E0C5F0C0E0C0F090F2E9122BB889828A835B
:2024E000E075F000C0E0C0F0740375F0001227367FFA122A8390F2E9E0A3F5F0E0C5F0124A
:202500002B0A90F2E9F0A3C5F0F0C5F0122B130224B312223A2205810581058105810581D7
:20252000740075F00078FD122A77F608A6F078FD122A77E60886F07B027C00122B2445F0EB
:202540007003022588801678FD122A77E60886F0122B0A18F608A6F0122B1380D178FD121C
:202560002A77E60886F079FA122A7C122A99C001C002122772C0E0C0F012275A1581158119
:20258000D007D000F602254778FD122A77E60886F079FA122A7C122A997400F7740075F060
:2025A0000079FA122A7C122A99E7C39430122AA97B04122AA0122AF9C0E0C0F0740175F00E
:2025C0000079F8122A7C122A99E7C39430D004D0034BC5F04CC5F0122AA97FFB022A92903A
:2025E000F2E6E0122AA97B3F122AA0122B4445F0700302260D90F004E0A3F5F0E0C5F0C009
:20260000E0C0F01227471581158112223A22058105810581058112264D78FB122A77F6082D
:20262000A6F012264D78FD122A77F608A6F0181818E60886F07B087C00122AF90846C5F0E0
:202640000846C5F015811581158115812205810581122772C0E0C0F012283C15811581C094
:20266000E0C0F012275A1581158178FD122A77F6122772C0E0C0F012283C15811581C0E0B0
:20268000C0F012275A1581158178FE122A77F618E6122AA9C0E0C0F01226CE158115817BCC
:2026A000047C00122AF978FD122A77F608E6122AA9C0E0C0F01226CE1581158178FE122A40
:2026C00077F618E60846122AA9158115812278FB122A77E6122AA9C0E0C0F01228B5158148
:2026E000158145F070030226F878FB122A77E6C39430122AA902273578FB122A77E6122A5E
:20270000A97B41122AA0122B3D45F0600CE6122AA97B46122AA0122B2B45F0700302272F8D
:2027200078FB122A77E6C39437122AA9022735740190F2DBF02223F42581F8122B95122916
:2027400009122B9502275178FB122A778682088683E0602D122760A380F778FB122A77E6B9
:202760003099FDC299F599B40A17740D80F2E430980C3098FDC298E599B40D02740A75F0E7
:20278000002278FB122A77E63099FDC299F5992274FFF5F030980A3098FDC298E59975F00E
:2027A000002278FC122A778604188603188683188682E4FDFE122772B408028003B47F273F
:2027C000ED4E60F11DBDFF011E7408122760742012276074081227608583F0E582122B136F
:2027E00085F083F58280CE122760F024F3600EA30DBD00010EED8EF0122B2470B8E4F0EDDD
:202800008EF02278FB122A778682088683E4FBFCFFE0A3B42D030FE0A3C39430B40A005071
:2028200012FA740A75F000122AB22AFBE5F03400FC80E4EB8CF0DF03022B1A2278FB122ACC
:2028400077E6C0E008E6C0E012288913D0F0D0E0500224E02278FB122A77E6C0E008E6C0D5
:20286000E012288E13D0F0D0E050E9242022D005D0061228B56009C006C00522D005D00633
:2028800012288E70F2C006C00590617A802A90415A802590217E802090007F801BD005D080
:2028A000069041461228B870CE9061661228B870C6C006C00590303978FB122A77E6B58384
:2028C00000400DB5820808E67006F5F0042240F6E4F5F02278FB122A77E690001FB47FDE10
:2028E00080E4D003D00412286EC004C00370E190207E80C478FB122A77E6C3940960C71434
:2029000060C4C3941660BF80C7122A50868208868308E4FEFFE07006122A50E4F022B42581
:2029200051A3E0B42D05430780A3E0B4300343074024D0B40A00500BCE75F00AA42EFEA362
:20294000E080EEE0B46413E60886F030F708430720122B1AA6F018F68003B4750543070A21
:202960008021B478054307108019B46F104307088011122A50F0A3122A50A38095B46262A1
:202980004307027A00C004C005C006C007AB0753031F7C00E60886F0122AC6A6F018F6EDC1
:2029A000D007D006D005D0042430B43A0040022407C0E00AE645F070CC122A50A902EF30BB
:2029C000E505742DF0A30A122A59D0E0F0A3D9FA0808EF30E7A1EAC39E509C7420F0A30A05
:2029E00080F4B4630DAA01122A50122A59E6F0A380DEB47331C082C08386820886837A002C
:202A0000E06004A30A80F98683188682122A50122A59122A50E0A3122A506004F0A380F2FE
:202A2000D005D00480AAB4691B86017A00E76004090A80F9122A50122A598601E76091F043
:202A400009A380F8F97A01122A50122A59E9809ECDC583CDCCC582CC22EE601A8FF020F7D5
:202A600015C002EAC39E500C742030F6027430F0A30A80EFD00222C82581C822C92581C9E8
:202A80007A0022D083D082CF2581F581CFC082C08322CF2581F581CF2229F9E5F03AFA226B
:202AA0007C00CB30E7011CCB2275F00030E70215F022FEEBA4FD8EF0ECA4FCEB8EF0A4C5A3
:202AC000F02C2DC5F022C002C001AAF0F97E007D007F11C3E933F9EA33FADF08F5F0E9D0C1
:202AE00001D00222ED33FDEE33FEC3ED9BF5F0EE9C40E0ADF0FED380DBBB000122C333C569
:202B0000F033C5F0DBF722122B0A04700205F022122B1314B4FF0215F022122B13F4C5F0DC
:202B2000F4C5F022122B774029801E122B7740227017801E122B7740107017800C122B7709
:202B400050108005122B8B6009E4F5F022122B8B60F7E4F5F00422122B8B40F680EB122BC0
:202B60008B40EF70E480EB122B8B40DD70E480D9122B8B50DD80D2C39BC5F09C20E7072026
:202B8000D207C345F02220D2F9D322C5F0C39C7003E5F09B2290F2EBE0A360F8E0FFA3E09F
:202BA000A3CF2582F582EF3583F58380EBFBE0CB22FCE0FBA3E0CC22FAE0F9A3E0CA2206A3
:202BC000F03DF042F00A0A38303531534243206E657720636F6D6D616E6473202870726581
:202BE0007373203F20666F722068656C70206F72207120746F207175697429000A0A3E3E2F
:202C0000000A0A48656C70204D656E750A41204153434949205461626C650A44204465630C
:202C2000324865780A522052656164204750494F320A5120517569740A4920692F6F2061AB
:202C40006464726573730A422042696E61727920696D6167650A3F2068656C70007072699E
:202C60006E7461626C6520415343494920636F64657328686578292C20652E672E20415369
:202C8000434949206F6620274127206973203431000A0A2020204D534200202020256400FB
:202CA0004C5342000A202025317820202000202020256300446563696D616C20746F2048B9
:202CC000657820636F6E766572746572000A0A456E74657220646563696D616C206E756DAE
:202CE0006265723D00446563202D3E20486578202D3E2042696E000A2564202D3E202578E3
:202D0000202D3E2025620052656164204750494F322028382D62697420696E7075742070B8
:202D20006F727429000A0A25303278202530386200692F6F206465636F64657220616464AD
:202D400072657373206D61646520627920504C44000A0A4C4344202020636F6D6D616E64DE
:202D60002077726974652020202020307830303030000A4C43442020206461746120777220
:202D80006974652020202020202020307830303031000A4C4344202020636F6D6D616E646C
:202DA0002072656164202020202020307830303032000A4C4344202020646174612072655F
:202DC0006164202020202020202020307830303033000A4750494F3120382D626974206FE6
:202DE000757470757420706F727420307830313030000A4750494F3220382D62697420696B
:202E00006E7075742020706F727420307830323030000A657870616E73696F6E20692F6F56
:202E200020737061636520202020203078303330302D3078303746460073656520686F77E8
:202E4000207265616C2070726F6772616D206C6F6F6B206C696B65000A0A656E74657220AA
:202E600061646472657373203D20000A0A4131352E2E2E2E2E2E2E2E2E2E2E2E4130204437
:172E8000372E2E2E2E2E4430000A2025303136622020253038620033
:20300000A5E5E0A5FDFF00000000000000000000000000000000000000000000FFFFFFFFA9
:103020003830353120545241494E4552204B495495
:20304000900200E030E15222C2AFC082C08390F291F0A3E5F0F0A3E5D0F0A353D0E7E8F04B
:20306000A3E9F0A3EAF0A3EBF0A3ECF0A3EDF0A3EEF0A3EFF0A3D0E0F0A3D0E0F090F28847
:20308000D0E0F090F287D0E0F090F2B3E581F090F2B4E0F5811237063275810D90573D79AF
:2030A000007AF07B4C7C02EB4C601CE493A3CAC583CAC9C582C9F0A3CAC583CAC9C582C997
:2030C0001BBBFFE31C80E090F2BDE4F01251A612001B80FB79027A0089828A83E0548070C7
:2030E000030230E70230D4221230D479007A00740189828A83F0221230D479007A0074382F
:2031000089828A83F01230D479007A00740F89828A83F01230E8740075F000C0E0C0F0744C
:203120000075F000C0E0C0F01231341581158115811581221230D478FB1255D2E6125604D5
:2031400090319602560D79007A0078F91255D2E6248089828A83F00231AA79007A0078F943
:203160001255D2E624C089828A83F00231AA79007A0078F91255D2E6249489828A83F00222
:2031800031AA79007A0078F91255D2E624D489828A83F00231AA823103006E3102005A3112
:2031A0000100463100000000AA31220581740078FE1255D2F678FE1255D2E6181818188680
:2031C0000108860275F0001255F489828A83E01256047B001255FB1256CB45F0700302324E
:2031E0001B800B78FE1255D2E604F61480C71230D479017A00C001C00278FC1255D2E61807
:20320000181818860108860275F0001255F489828A83E0D083D082F00231E31581227400C0
:2032200075F000C0E0C0F0740175F000C0E0C0F01231341581158115811581740090F24C9E
:20324000F090F24CE01256047B141255FB1256A245F0700302328B800C90F24CE00490F242
:203260004CF01480DC1230D490F24CE0794D7AF21256041255F4C001C00279037A00898261
:203280008A83E0D083D082F00232591230E8740075F000C0E0C0F0740075F000C0E0C0F0A3
:2032A0001231341581158115811581794D7AF2E98AF0C0E0C0F01231AB1581158174007557
:2032C000F000C0E0C0F0740175F000C0E0C0F0123134158115811581158122740075F000BA
:2032E000C0E0C0F0740075F000C0E0C0F01231341581158115811581740090F24CF090F2D2
:203300004CE01256047B141255FB1256A245F07003023348800C90F24CE00490F24CF014E5
:2033200080DC1230D490F24CE0794D7AF21256041255F4C001C00279037A0089828A83E003
:20334000D083D082F00233161230E8740075F000C0E0C0F0740175F000C0E0C0F012313499
:203360001581158115811581794D7AF2E98AF0C0E0C0F01231AB15811581740075F000C05D
:20338000E0C0F0740075F000C0E0C0F01231341581158115811581221230D479017A007801
:2033A000FB1255D2E689828A83F02279917AF2E98AF02402C5F03400C5F0F9AAF089828A04
:2033C00083E090F266F090F266E090F267F090F266E0548070030233E8740190F266F0E5B3
:2033E00090547FF5900233F4740090F266F0E5904480F59090F266E0542070030234087451
:203400000190F267F002340E740090F267F079737AF2E98AF0C0E0C0F0741075F0F0C0E0BD
:20342000C0F079917AF2E98AF0F9AAF089828A83E075F000C0E0C0F079917AF2E98AF024C6
:2034400001C5F03400C5F0F9AAF089828A83E075F000C0E0C0F090F266E075F000C0E0C000
:20346000F090F267E075F000C0E0C0F0740675F00012534B7FF41255DE740075F000C0E01E
:20348000C0F0740075F000C0E0C0F0123134158115811581158179737AF2E98AF0C0E0C069
:2034A000F01231AB158115812279737AF2E98AF0C0E0C0F0742B75F0F0C0E0C0F079917A0D
:2034C000F2E98AF02402C5F03400C5F0F9AAF089828A83E075F000C0E0C0F079917AF2E934
:2034E0008AF0240BC5F03400C5F0F9AAF089828A83E075F000C0E0C0F079917AF2E98AF06C
:20350000240CC5F03400C5F0F9AAF089828A83E075F000C0E0C0F0740575F00012534B7F90
:20352000F61255DE740075F000C0E0C0F0740075F000C0E0C0F012313415811581158115B0
:203540008179737AF2E98AF0C0E0C0F01231AB158115812279917AF2E98AF02403C5F034BA
:2035600000C5F0F9AAF089828A83E0F50A79917AF2E98AF02404C5F03400C5F0F9AAF08951
:20358000828A83E0F50B79917AF2E98AF02405C5F03400C5F0F9AAF089828A83E0F50C7917
:2035A000917AF2E98AF02406C5F03400C5F0F9AAF089828A83E0F50D79737AF2E98AF0C0DB
:2035C000E0C0F0744275F0F0C0E0C0F0E50A75F000C0E0C0F0E50B75F000C0E0C0F0E50CC6
:2035E00075F000C0E0C0F0E50D75F000C0E0C0F0740675F00012534B7FF41255DE7400753F
:20360000F000C0E0C0F0740075F000C0E0C0F0123134158115811581158179737AF2E98AA7
:20362000F0C0E0C0F01231AB158115812279917AF2E98AF02407C5F03400C5F0F9AAF08950
:20364000828A83E0F50A79917AF2E98AF02408C5F03400C5F0F9AAF089828A83E0F50B7955
:20366000917AF2E98AF02409C5F03400C5F0F9AAF089828A83E0F50C79917AF2E98AF02496
:203680000AC5F03400C5F0F9AAF089828A83E0F50D79737AF2E98AF0C0E0C0F0745B75F0B6
:2036A000F0C0E0C0F0E50A75F000C0E0C0F0E50B75F000C0E0C0F0E50C75F000C0E0C0F0DB
:2036C000E50D75F000C0E0C0F0740675F00012534B7FF41255DE740075F000C0E0C0F0745F
:2036E0000075F000C0E0C0F0123134158115811581158179737AF2E98AF0C0E0C0F01231F8
:20370000AB158115812290F2B5E075F0007B007C001256C245F0700302371E1233AB90F2A2
:20372000B5E075F0007B017C001256C245F070030237361234A990F2B5E075F0007B027CF2
:20374000001256C245F0700302374E12355490F2B5E075F0007B037C001256C245F070032D
:2037600002376612362D740075F004C0E0C0F079917AF2E98AF0F9AAF089828A83E075F03F
:2037800000C0E0C0F012537A158115811581158190F2B3E0F50A90F26EE070030237BFE56E
:2037A0000A2402F50A90F28BE0A3F5F0E0C5F090F287F0A3C5F0F0C5F0740090F26EF0E5A1
:2037C0000A90F2B3F0A80A860A740075F000C0E0C0F0740175F000C0E0C0F0123134158118
:2037E00015811581158179737AF2E98AF0C0E0C0F0747475F0F0C0E0C0F090F287E0A3F5EE
:20380000F0E0C5F0C0E0C0F090F28712573689828A83E075F000C0E0C0F090F2B3E075F004
:2038200000C0E0C0F0E50A75F000C0E0C0F0740675F00012534B7FF41255DE79737AF2E90C
:203840008AF0C0E0C0F01231AB158115812290F262E01256047B111255FB1256C245F07075
:20386000030238F07403F5087430F5091230E8740190F26EF090F287E0A3F5F0E0C5F090F0
:20388000F28BF0A3C5F0F0C5F0903048C082C0839080137402F0A3D0E0F0D0E0A3F090F2A0
:2038A000B4E581F090F2B3E0F58190F287E0C0E0A3E0C0E090F291E0C0E0A3E0C0E0A3E08E
:2038C000C0E07F08A3E0C0E0DFFAA3E0C0E0A3E0C0E0D082D083D007D006D005D004D003B1
:2038E000D002D001D000D0D053D0E7D0F0D0E0222274FF90F262F0740090F264F074019061
:20390000F26BF0740090F263F090F263E01256047B071255FB1256A245F070030239E280AD
:203920000C90F263E00490F263F01480DC740075F001C0E0C0F090F26BE0F4125604C0E076
:20394000C0F012537A1581158115811581740075F002C0E0C0F01253591581158190F26683
:20396000F0740090F265F090F265E01256047B041255FB1256A245F070030239CC800C9023
:20398000F265E00490F265F01480DC90F266E0548075F0007B007C001256C245F0700302D9
:2039A00039AD90F264E090F262F00239B790F264E00490F264F01490F266E075F0007B0138
:2039C0007C0012566990F266F002397F90F26BE01256047B011255FB12566990F26BF00241
:2039E000392190F262E012560422740090F267F01238F11256047BFF1255FB1256CB45F0E3
:203A0000600E90F2B6E075F0007B007C001256C245F07003023A4C90F267E00490F267F0C4
:203A200075F0007B967C001256E545F0600E90F2B6E075F0007B007C001256C245F070035E
:203A4000023A49740190F2B6F00239F0740A75F000C0E0C0F012539A158115811238F1126E
:203A600056047BFF1255FB1256C245F07003023A7A740090F2B6F0023A5C90F262E0125628
:203A8000047B101255FB1256A245F07003023AA790F262E079007AF01256041255F4898227
:203AA0008A83E090F262F02290F26DE07003023AFB740075F001C0E0C0F0747F75F0FFC069
:203AC000E0C0F012537A1581158115811581740175F000C0E0C0F012539A15811581740056
:203AE00075F001C0E0C0F074FF75F000C0E0C0F012537A15811581158115812290F262E0CB
:203B00001256047B101255FB1256C245F07003023C15123AA890F287E0A3F5F0E0C5F07BB2
:203B2000007C801256D545F07003023B3C740075F08090F287F0A3C5F0F0C5F07400F5086B
:203B400012321E79737AF2E98AF0C0E0C0F0748B75F0F0C0E0C0F090F287E0A3F5F0E0C53E
:203B6000F0C0E0C0F090F28712573689828A83E075F000C0E0C0F090F287E0A3F5F0E0C59A
:203B8000F02401C5F03400C5F0F9AAF089828A83E075F000C0E0C0F090F287E0A3F5F0E0E1
:203BA000C5F02402C5F03400C5F0F9AAF089828A83E075F000C0E0C0F090F287E0A3F5F0DB
:203BC000E0C5F02403C5F03400C5F0F9AAF089828A83E075F000C0E0C0F0740775F0001259
:203BE000534B7FF21255DE79737AF2E98AF0C0E0C0F01231AB1581158190F287E0A3F5F0DB
:203C0000E0C5F02404C5F03400C5F090F287F0A3C5F0F0C5F02290F262E01256047B16125E
:203C200055FB1256C245F07003023CFE123AA87401F508740075F09090F287F0A3C5F0F016
:203C4000C5F01230E8740075F000C0E0C0F0740175F000C0E0C0F0123134158115811581F9
:203C6000158174A475F0F0C0E0C0F01231AB1581158112321E740075F000C0E0C0F07401D7
:203C800075F000C0E0C0F0123134158115811581158179737AF2E98AF0C0E0C0F074B475F8
:203CA000F0F0C0E0C0F090F287E0A3F5F0E0C5F0C0E0C0F090F28712573689828A83E07569
:203CC000F000C0E0C0F0740475F00012534B7FF81255DE79737AF2E98AF0C0E0C0F012310D
:203CE000AB15811581740075F00090F28FF0A3C5F0F0C5F07430F509746090F2B3F02290C9
:203D0000F262E01256047B1A1255FB1256C245F07003023D61123AA81230E8740075F000A3
:203D2000C0E0C0F0740175F000C0E0C0F0123134158115811581158174C175F0F0C0E0C050
:203D4000F01231AB1581158112321E123D627402F508740075F00090F28FF0A3C5F0F0C5EC
:203D6000F02279737AF2E98AF0C0E0C0F074CE75F0F0C0E0C0F090F287E0A3F5F0E0C5F039
:203D8000C0E0C0F0740375F00012534B7FFA1255DE79737AF2E98AF0C0E0C0F01231AB157B
:203DA0008115812290F262E01256047B141255FB1256C245F07003023E53123AA87401F5E6
:203DC00008740075F000C0E0C0F0740175F000C0E0C0F0123134158115811581158174D471
:203DE00075F0F0C0E0C0F01231AB1581158112321E79737AF2E98AF0C0E0C0F074E575F0D9
:203E0000F0C0E0C0F090F287E0A3F5F0E0C5F0C0E0C0F090F28712573689828A83E075F007
:203E200000C0E0C0F0740475F00012534B7FF81255DE79737AF2E98AF0C0E0C0F01231ABF0
:203E400015811581740075F00090F28FF0A3C5F0F0C5F02290F262E01256047B181255FB18
:203E60001256C245F0600DE5081256047B011255FB1256C245F07003023F6D123AA8740057
:203E800075F000C0E0C0F0740175F000C0E0C0F0123134158115811581158179737AF2E933
:203EA0008AF0C0E0C0F074F275F0F0C0E0C0F090F287E0A3F5F0E0C5F0C0E0C0F090F287CE
:203EC00012573689828A83E075F000C0E0C0F0740475F00012534B7FF81255DE79737AF2F5
:203EE000E98AF0C0E0C0F01231AB1581158112321E90F287E0A3F5F0E0C5F012568890F21B
:203F000087F0A3C5F0F0C5F012569179737AF2E98AF0C0E0C0F0740175F0F1C0E0C0F0907E
:203F2000F287E0A3F5F0E0C5F0C0E0C0F090F28712573689828A83E075F000C0E0C0F074F2
:203F40000475F00012534B7FF81255DE79737AF2E98AF0C0E0C0F01231AB158115817400F3
:203F600075F00090F28FF0A3C5F0F0C5F02290F262E01256047B191255FB1256C245F060D7
:203F80000DE5081256047B011255FB1256C245F07003024087123AA8740075F000C0E0C015
:203FA000F0740075F000C0E0C0F0123134158115811581158179737AF2E98AF0C0E0C0F00E
:203FC000740E75F0F1C0E0C0F090F287E0A3F5F0E0C5F0C0E0C0F090F28712573689828A26
:203FE00083E075F000C0E0C0F0740475F00012534B7FF81255DE79737AF2E98AF0C0E0C045
:20400000F01231AB158115811232DB90F287E0A3F5F0E0C5F012569190F287F0A3C5F0F037
:20402000C5F012568879737AF2E98AF0C0E0C0F0741B75F0F1C0E0C0F090F287E0A3F5F02A
:20404000E0C5F0C0E0C0F090F28712573689828A83E075F000C0E0C0F0740475F0001253E4
:204060004B7FF81255DE79737AF2E98AF0C0E0C0F01231AB15811581740075F00090F28F2A
:20408000F0A3C5F0F0C5F02278FB1255D2E61256047B091255FB1256B245F0600CE6125624
:2040A000047B101255FB1256A245F070030240C490F262E02437125604C0E0C0F01233989F
:2040C0001581158178FB1255D2E61256047B001255FB1256BB45F0600CE61256047B0A122C
:2040E00055FB1256A245F0700302410090F262E02430125604C0E0C0F0123398158115819E
:204100002290F262E01256047B001255FB1256BB45F0600F90F262E01256047B0F1255FB8D
:204120001256A945F07003024A91E5081256047B011255FB1256C245F070030242AC123AA4
:20414000A890F262E0125604C0E0C0F01240881581158190F28712573689828A83E090F20F
:2041600066F090F266E075F0007B047C0012566990F266F090F266E054F090F266E090F2C2
:204180006212572B4B90F266F090F28712573690F266E089828A83F090F28FE0A3F5F0E035
:2041A000C5F012568890F28FF0A3C5F0F0C5F07B017C001256E545F070030242AC74007596
:2041C000F00090F28FF0A3C5F0F0C5F0740075F000C0E0C0F0740175F000C0E0C0F012315B
:2041E00034158115811581158179737AF2E98AF0C0E0C0F0742875F0F1C0E0C0F090F287DD
:20420000E0A3F5F0E0C5F0C0E0C0F090F28712573689828A83E075F000C0E0C0F07404750F
:20422000F00012534B7FF81255DE79737AF2E98AF0C0E0C0F01231AB1581158112321E900B
:20424000F287E0A3F5F0E0C5F012568890F287F0A3C5F0F0C5F012569179737AF2E98AF04E
:20426000C0E0C0F0743775F0F1C0E0C0F090F287E0A3F5F0E0C5F0C0E0C0F090F2871257D5
:204280003689828A83E075F000C0E0C0F0740475F00012534B7FF81255DE79737AF2E98A27
:2042A000F0C0E0C0F01231AB15811581E5081256047B021255FB1256C245F0700302434F06
:2042C000123AA890F262E0125604C0E0C0F01240881581158190F287E0A3F5F0E0C5F090CE
:2042E000F26FF0A3C5F0F0C5F090F26FE0A3F5F0E0C5F07B047C0012566990F26FF0A3C56D
:20430000F0F0C5F090F26FE0A3F5F0E0C5F054F0C5F054FFC5F090F26FF0A3C5F0F0C5F03B
:2043200090F26FE0A3F5F0E0C5F090F26212572B4B90F26FF0A3C5F0F0C5F090F26FE0A37A
:20434000F5F0E0C5F090F287F0A3C5F0F0C5F0E5081256047B041255FB1256C245F07003E1
:20436000024366124CB3E5081256047B051255FB1256C245F070030244D5123AA890F26281
:20438000E0125604C0E0C0F01240881581158190F28DE0A3F5F0E0C5F090F26FF0A3C5F036
:2043A000F0C5F090F26FE0A3F5F0E0C5F07B047C0012566990F26FF0A3C5F0F0C5F090F23E
:2043C0006FE0A3F5F0E0C5F054F0C5F054FFC5F090F26FF0A3C5F0F0C5F090F26FE0A3F529
:2043E000F0E0C5F090F26212572B4B90F26FF0A3C5F0F0C5F090F26FE0A3F5F0E0C5F09019
:20440000F28DF0A3C5F0F0C5F090F28FE0A3F5F0E0C5F012568890F28FF0A3C5F0F0C5F034
:204420007B047C001256E545F070030244D590F287E0A3F5F0E0C5F02401C5F03400C5F0A8
:20444000FBACF090F28DE0A3F5F0E0C5F0C39BC5F09CC5F090F26FF0A3C5F0F0C5F090F2F5
:204460006FE0A3F5F0E0C5F090F266F090F28712573690F266E089828A83F012321E797332
:204480007AF2E98AF0C0E0C0F0744475F0F1C0E0C0F090F287E0A3F5F0E0C5F0C0E0C0F049
:2044A00090F28712573689828A83E075F000C0E0C0F0740475F00012534B7FF81255DE79E5
:2044C000737AF2E98AF0C0E0C0F01231AB158115817401F508E5081256047B061255FB1270
:2044E00056C245F070030246A9123AA890F262E0125604C0E0C0F01240881581158190F20F
:204500008DE0A3F5F0E0C5F090F26FF0A3C5F0F0C5F090F26FE0A3F5F0E0C5F07B047C004A
:2045200012566990F26FF0A3C5F0F0C5F090F26FE0A3F5F0E0C5F054F0C5F054FFC5F0904D
:20454000F26FF0A3C5F0F0C5F090F26FE0A3F5F0E0C5F090F26212572B4B90F26FF0A3C513
:20456000F0F0C5F090F26FE0A3F5F0E0C5F090F28DF0A3C5F0F0C5F090F28FE0A3F5F0E063
:20458000C5F012568890F28FF0A3C5F0F0C5F07B047C001256E545F070030246A990F28D88
:2045A000E0A3F5F0E0C5F090F28712572FC39BC5F09CC5F090F26FF0A3C5F0F0C5F090F299
:2045C0006FE0A3F5F0E0C5F07B007C001256B245F07003024640740075F00090F271F0A3CF
:2045E000C5F0F0C5F090F271E0A3F5F0E0C5F090F26F12572F1256A245F07003024640802E
:204600001C90F271E0A3F5F0E0C5F012568890F271F0A3C5F0F0C5F012569180C890F28774
:20462000E0A3F5F0E0C5F090F27112572F2BC5F03CC5F0F9AAF0740089828A83F0024601C9
:2046400012321E79737AF2E98AF0C0E0C0F0745175F0F1C0E0C0F090F287E0A3F5F0E0C56C
:20466000F0C0E0C0F090F28712573689828A83E075F000C0E0C0F0740475F00012534B7F99
:20468000F81255DE79737AF2E98AF0C0E0C0F01231AB158115817401F508740075F00090DD
:2046A000F28FF0A3C5F0F0C5F0E5081256047B071255FB1256C245F0700302489D123AA8A2
:2046C00090F262E0125604C0E0C0F01240881581158190F28DE0A3F5F0E0C5F090F26FF067
:2046E000A3C5F0F0C5F090F26FE0A3F5F0E0C5F07B047C0012566990F26FF0A3C5F0F0C515
:20470000F090F26FE0A3F5F0E0C5F054F0C5F054FFC5F090F26FF0A3C5F0F0C5F090F26FEB
:20472000E0A3F5F0E0C5F090F26212572B4B90F26FF0A3C5F0F0C5F090F26FE0A3F5F0E0A2
:20474000C5F090F28DF0A3C5F0F0C5F090F28FE0A3F5F0E0C5F012568890F28FF0A3C5F051
:20476000F0C5F07B047C001256E545F0700302489D90F28DE0A3F5F0E0C5F090F26FF0A32D
:20478000C5F0F0C5F090F26FE0A3F5F0E0C5F054FFC5F05400C5F090F266F090F26FE0A374
:2047A000F5F0E0C5F07B087C0012567790F26FF0A3C5F0F0C5F090F267F090F267E075F0BC
:2047C000007B057C0012566990F267F090F267E0440190F267F090F28712573690F267E0DB
:2047E00089828A83F090F287E0A3F5F0E0C5F02401C5F03400C5F0F9AAF090F266E0898282
:204800008A83F012321E79737AF2E98AF0C0E0C0F0745E75F0F1C0E0C0F090F287E0A3F535
:20482000F0E0C5F0C0E0C0F090F28712573689828A83E075F000C0E0C0F0740475F000125F
:20484000534B7FF81255DE79737AF2E98AF0C0E0C0F01231AB158115817401F50890F28D58
:20486000E0A3F5F0E0C5F090F28712572FC39BC5F09CC5F0C0E0C0F01253B7158115817B23
:20488000007C081256BB45F0700302489D743F75F000C0E0C0F012339815811581E5081272
:2048A00056047B081255FB1256C245F07003024A91123AA890F262E0125604C0E0C0F01284
:2048C00040881581158190F28DE0A3F5F0E0C5F090F26FF0A3C5F0F0C5F090F26FE0A3F591
:2048E000F0E0C5F07B047C0012566990F26FF0A3C5F0F0C5F090F26FE0A3F5F0E0C5F05447
:20490000F0C5F054FFC5F090F26FF0A3C5F0F0C5F090F26FE0A3F5F0E0C5F090F2621257D1
:204920002B4B90F26FF0A3C5F0F0C5F090F26FE0A3F5F0E0C5F090F28DF0A3C5F0F0C5F039
:2049400090F28FE0A3F5F0E0C5F012568890F28FF0A3C5F0F0C5F07B047C001256E545F0DE
:204960007003024A9190F28DE0A3F5F0E0C5F090F26FF0A3C5F0F0C5F090F26FE0A3F5F0A4
:20498000E0C5F054FFC5F05400C5F090F266F090F26FE0A3F5F0E0C5F07B087C00125677CD
:2049A00090F26FF0A3C5F0F0C5F090F267F090F267E075F0007B057C0012566990F267F06C
:2049C00090F267E0441190F267F090F28712573690F267E089828A83F090F287E0A3F5F0F6
:2049E000E0C5F02401C5F03400C5F0F9AAF090F266E089828A83F012321E79737AF2E98ACF
:204A0000F0C0E0C0F0746B75F0F1C0E0C0F090F287E0A3F5F0E0C5F0C0E0C0F090F2871260
:204A2000573689828A83E075F000C0E0C0F0740475F00012534B7FF81255DE79737AF2E9B2
:204A40008AF0C0E0C0F01231AB158115817401F50890F28DE0A3F5F0E0C5F090F287125782
:204A60002FC39BC5F09CC5F0C0E0C0F01253B7158115817B007C081256BB45F07003024AF5
:204A800091743F75F000C0E0C0F0123398158115812290F262E01256047B151255FB125668
:204AA000C245F07003024B21123AA812321EA809860A08860B08860C08860D79737AF2E978
:204AC0008AF0C0E0C0F0747875F0F1C0E0C0F0E50975F000C0E0C0F0E50A75F000C0E0C023
:204AE000F0E50B75F000C0E0C0F0E50C75F000C0E0C0F0E50D75F000C0E0C0F0740775F0F4
:204B00000012534B7FF21255DE79737AF2E98AF0C0E0C0F01231AB15811581E5092404F5FF
:204B20000922740075F001C0E0C0F0747F75F0FFC0E0C0F012537A158115811581158174CE
:204B40006475F000C0E0C0F012539A15811581740075F001C0E0C0F074FF75F000C0E0C0AF
:204B6000F012537A158115811581158122740075F004C0E0C0F074FF75F000C0E0C0F01285
:204B8000537A1581158115811581747FF59090F26CE01256047BAA1255FB1256CB45F070DF
:204BA00003024BB374AA90F26CF0124B22740190F26DF0740075F004C0E0C0F0740075F01D
:204BC00000C0E0C0F012537A158115811581158174FFF5902290F262E01256047B1312550F
:204BE000FB1256C245F07003024C73123AA890F2B5E00490F2B5F01490F2B5E075F0007BE6
:204C0000037C001256E545F07003024C13740090F2B5F090F2B5E075F0007B007C00125649
:204C2000C245F07003024C2B1233AB90F2B5E075F0007B017C001256C245F07003024C43CA
:204C40001234A990F2B5E075F0007B027C001256C245F07003024C5B12355490F2B5E0754E
:204C6000F0007B037C001256C245F07003024C7312362D2290F262E01256047B171255FBFC
:204C80001256C245F0600DE5081256047B011255FB1256C245F07003024CB2123AA87404D3
:204CA000F508749375F0F1C0E0C0F01231AB158115812290F262E01256047B0A1255FB12E5
:204CC00056C245F07003024DF11230E8740075F000C0E0C0F0740175F000C0E0C0F0123114
:204CE000341581158115811581749775F0F1C0E0C0F01231AB15811581740075F00290F200
:204D00006FF0A3C5F0F0C5F090F26FE0A3F5F0E0C5F07B007C001256B245F07003024D8AB7
:204D2000801C90F26FE0A3F5F0E0C5F012569190F26FF0A3C5F0F0C5F012568880CA90F256
:204D400087E0A3F5F0E0C5F090F26F12572F2BC5F03CC5F0F9AAF090F287E0A3F5F0E0C5CC
:204D6000F090F26F12572F2BC5F03CC5F0C39401C5F09400C5F0C001C002F9AAF089828AE8
:204D800083E0D083D082F0024D2290F287125736740089828A83F012321E79737AF2E98A59
:204DA000F0C0E0C0F074A775F0F1C0E0C0F090F287E0A3F5F0E0C5F0C0E0C0F090F2871281
:204DC000573689828A83E075F000C0E0C0F0740475F00012534B7FF81255DE79737AF2E90F
:204DE0008AF0C0E0C0F01231AB158115817401F50890F262E01256047B0D1255FB1256C219
:204E000045F07003024F211230E8740075F000C0E0C0F0740175F000C0E0C0F0123134156F
:204E20008115811581158174B475F0F1C0E0C0F01231AB15811581740075F00090F26FF08D
:204E4000A3C5F0F0C5F090F26FE0A3F5F0E0C5F07B007C021256A245F07003024EC7801C09
:204E600090F26FE0A3F5F0E0C5F012568890F26FF0A3C5F0F0C5F012569180CA90F287E04A
:204E8000A3F5F0E0C5F090F26F12572F2BC5F03CC5F0F9AAF090F287E0A3F5F0E0C5F09072
:204EA000F26F12572F2BC5F03CC5F02401C5F03400C5F0C001C002F9AAF089828A83E0D087
:204EC00083D082F0024E6012321E79737AF2E98AF0C0E0C0F074C375F0F1C0E0C0F090F291
:204EE00087E0A3F5F0E0C5F0C0E0C0F090F28712573689828A83E075F000C0E0C0F0740411
:204F000075F00012534B7FF81255DE79737AF2E98AF0C0E0C0F01231AB158115817401F531
:204F20000890F262E01256047B0B1255FB1256C245F07003024F7590F262E0125604C0E0E9
:204F4000C0F01240881581158112321E74D075F0F1C0E0C0F01231AB158115817405F508BF
:204F6000740075F00090F28FF0A3C5F0F0C5F074FF90F262F090F262E01256047B081255F9
:204F8000FB1256C245F07003024F9E12321E74D975F0F1C0E0C0F01231AB1581158190F264
:204FA00062E01256047B0C1255FB1256C245F0700302502390F262E0125604C0E0C0F01281
:204FC00040881581158112321E79737AF2E98AF0C0E0C0F074EA75F0F1C0E0C0F090F28763
:204FE000E0A3F5F0E0C5F0C0E0C0F0740375F00012534B7FFA1255DE79737AF2E98AF0C09F
:20500000E0C0F01231AB158115817406F508740075F00090F28FF0A3C5F0F0C5F074FF9095
:20502000F262F090F262E01256047B091255FB1256C245F0700302507290F26DE0640190BC
:20504000F26DF012321E90F26DE0700302506274F175F0F1C0E0C0F01231AB158115810282
:20506000507274F975F0F1C0E0C0F01231AB1581158190F262E01256047B0E1255FB1256BE
:20508000C245F070030250C690F262E0125604C0E0C0F01240881581158112321E740275BB
:2050A000F0F2C0E0C0F01231AB158115817407F508740075F00090F28FF0A3C5F0F0C5F055
:2050C00074FF90F262F090F262E01256047B0F1255FB1256C245F0700302511A90F262E06A
:2050E000125604C0E0C0F01240881581158112321E740B75F0F2C0E0C0F01231AB158115CD
:20510000817408F508740075F00090F28FF0A3C5F0F0C5F074FF90F262F02290F262E0127F
:2051200056047B121255FB1256C245F070030251A57407F508903048C082C08390801374C0
:2051400002F0A3D0E0F0D0E0A3F0123AA890F2B4E581F090F2B3E0F58190F287E0C0E0A3A0
:20516000E0C0E090F291E0C0E0A3E0C0E0A3E0C0E07F08A3E0C0E0DFFAA3E0C0E0A3E0C0ED
:20518000E0D082D083D007D006D005D004D003D002D001D000D0D053D0E7D0F0D0E0C28A88
:2051A000D2AAD2AF3222740075F004C0E0C0F074FF75F000C0E0C0F012537A158115811529
:2051C000811581747FF59074C875F000C0E0C0F012539A158115811230F7124B6D74007538
:2051E000F000C0E0C0F0740075F000C0E0C0F01231341581158115811581741575F0F2C0D7
:20520000E0C0F01231AB15811581740075F000C0E0C0F0740175F000C0E0C0F01231341505
:2052200081158115811581740075F09090F287F0A3C5F0F0C5F07430F509740075F00090C1
:20524000F28FF0A3C5F0F0C5F074FFF5907401F50879737AF2E98AF0C0E0C0F0742675F06C
:20526000F2C0E0C0F090F287E0A3F5F0E0C5F0C0E0C0F090F28712573689828A83E075F091
:2052800000C0E0C0F0740475F00012534B7FF81255DE79737AF2E98AF0C0E0C0F01231AB7C
:2052A00015811581740090F2B2F0740190F2B1F0740090F2B6F0746090F2B3F0740090F207
:2052C0006EF0740090F2B5F01239EA743375F0F2C0E0C0F090F262E0125604C0E0C0F09042
:2052E000F287E0A3F5F0E0C5F0C0E0C0F0740075F00079917AF21255F489828A83E075F0E1
:2053000000C0E0C0F0740475F00012533A7FF81255DE123AFC123CFF123C16123DA41241C6
:2053200001123F6E123E5412384E124A92124C7412511B124BD50252C82223F42581F812FC
:20534000571312546412571302543323F42581F886820886830802546478FB1255D28682D0
:20536000088683E075F0002278FB1255D28682088683E0F5F0A3E0C5F02278F91255D286A1
:205380008208868308E6F02278F91255D2868208868308E608F0A3E6F02278FB1255D28604
:2053A00003088604BB0004BC00012279E5A3D9FD1BBBFFF01C80F478FB1255D2E60886F07E
:2053C00030F73A02569878F91255D28603088604088605088606ED8EF01256F5401CED8EF1
:2053E000F02278F91255D28603088604088605088606ED8EF01256F540E4EB8CF02278FBC7
:205400001255D2860308860475F0FE74017F001256D5600575F001E422EF0FF5F0A41256E4
:20542000D570F6EF1475F0002278FB1255D28682088683E0602D125442A380F778FB1255D9
:20544000D2E63099FDC299F599B40A17740D80F2E430980C3098FDC298E599B40D02740A87
:2054600075F000221255AB868208868308E4FEFFE070061255ABE4F022B42551A3E0B42DA5
:2054800005430780A3E0B4300343074024D0B40A00500BCE75F00AA42EFEA3E080EEE0B4AA
:2054A0006413E60886F030F708430720125698A6F018F68003B4750543070A8021B47805FD
:2054C0004307108019B46F1043070880111255ABF0A31255ABA38095B462624307027A0016
:2054E000C004C005C006C007AB0753031F7C00E60886F0125636A6F018F6EDD007D006D0E3
:2055000005D0042430B43A0040022407C0E00AE645F070CC1255ABA902EF30E505742DF0AB
:20552000A30A1255B4D0E0F0A3D9FA0808EF30E7A1EAC39E509C7420F0A30A80F4B4630DD6
:20554000AA011255AB1255B4E6F0A380DEB47331C082C08386820886837A00E06004A30A3B
:2055600080F986831886821255AB1255B41255ABE0A31255AB6004F0A380F2D005D0048023
:20558000AAB4691B86017A00E76004090A80F91255AB1255B48601E76091F009A380F8F9B8
:2055A0007A011255AB1255B4E9809ECDC583CDCCC582CC22EE601A8FF020F715C002EAC3D7
:2055C0009E500C742030F6027430F0A30A80EFD00222C82581C822C92581C97A0022D083F2
:2055E000D082CF2581F581CFC082C08322CF2581F581CF2229F9E5F03AFA227C00CB30E771
:20560000011CCB2275F00030E70215F022FDE493A3FEE493A3FF4E7009E493FE740193FF6A
:20562000800BE493A3B5050BE493B5F0068F838E82E473A380D8C002C001AAF0F97E007D59
:20564000007F11C3E933F9EA33FADF08F5F0E9D001D00222ED33FDEE33FEC3ED9BF5F0EEF7
:205660009C40E0ADF0FED380DBBB000122C333C5F033C5F0DBF722BB000122C3C5F013C512
:20568000F013DBF72212568804700205F02212569114B4FF0215F022125691F4C5F0F4C552
:2056A000F0221256F54029801E1256F540227017801E1256F540107017800C1256F5501013
:2056C00080051257096009E4F5F02212570960F7E4F5F0042212570940F680EB1257094002
:2056E000EF70E480EB12570940DD70E480D912570950DD80D2C39BC5F09C20E70720D20719
:20570000C345F02220D2F9D322C5F0C39C7003E5F09B2290F2BDE0A360F8E0FFA3E0A3CF88
:205720002582F582EF3583F58380EBFBE0CB22FCE0FBA3E0CC22FAE0F9A3E0CA2200040863
:205740000C0105090D02060A0E03070B0F413D2530327820423D2530327820632530316257
:2057600020616325303162005053573D2530327820445054523D2530327825303278005240
:20578000302D333A253032782025303278202530327820253032780052342D373A25303238
:2057A0007820253032782025303278202530327800253034783A253032782053503D253085
:2057C00032783A2530327800253034783A253032782025303278202530327820253032784F
:2057E00000707573682053544550207C2052554E0025303478205B253032785D20006E6511
:2058000077206C6F636174696F6E00253034783E00656E7465722068657820636F646520FB
:20582000200025303478205B253032785D200025303478205B253032785D202020002530C3
:205840003478205B253032785D200025303478205B253032785D200025303478205B2530DC
:2058600032785D200025303478205B253032785D2020200025303478205B253032785D20D1
:205880000025303478205B253032785D200025303478205B253032785D20002530347820F7
:2058A0005B253032785D200025303478205B253032785D200020253032783A2025303278A1
:2058C00020253032782025303278202530327800616C7400696E73657274206279746520A1
:2058E0002020200025303478205B253032785D200064656C657465206279746520202000A9
:2059000025303478205B253032785D20006A756D7020746F3D005265762E312E3020322F28
:20592000372F3230303900253034782D3E0042656570204F4E0042656570204F46460041D9
:205940004A4D5020746F3D004143414C4C20746F3D003830353120545241494E4552204B15
:2059600049540025303478205B253032785D20000A6B6579203D2025642050433D253034C0
:095980007820413D253032780009
:00000001FF
